:040000000AEF12F001
:1000080000C017F001C016F002C015F06F0084FFA1
:1000180018F06F0088FF19F03901A3A7D4D093A76F
:10002800D2D05BEC0DF000C048F03D01F9AB11D027
:10003800F99B010E1E01D225006E000ED321016E20
:10004800600001F0D2FE600005F0D3FE6F00A0F75B
:1000580048F03D01F9A711D0010E1E01D225006E0E
:10006800000ED321016E600001F0D2FE600005F0A1
:10007800D3FE5BEC0DF000C048F03D01F9A511D0AE
:10008800010E1E01D225006E000ED321016E600004
:1000980001F0D2FE600005F0D3FE5BEC0DF000C06D
:1000A80048F0510E0001D125E16E000ED221E26E1A
:1000B8006F0087FFE1FF6F008BFFE2FF600023F115
:1000C800E6FF400E495C016E000E4A58026E600061
:1000D80005F01FFF600009F020FF800E006E800E03
:1000E8000218005C02E1015000081AE2800E1F01AC
:1000F8002019006E800E1D0A005C02E14C0E1F5D87
:100108000FE2820E1F25E16E010E2021E26E6F00C4
:1001180087FFE1FF6F008BFFE2FF600023F1E6FF3E
:10012800010E4924006E000E4A20016E00C049F0FD
:1001380001C04AF0010E0001D125006E000ED22147
:10014800016E00C0D1F001C0D2F030D00001000E25
:10015800006ED251005C02E1D1513F0810E2BC8A26
:1001680039019397010E0001D76F000ED86FD16B3C
:10017800D26B39019397010E1A6E000E1B6E23D0B5
:10018800000E006E0001D251005C02E1D1513F081F
:100198000CE2BC8A39019397010E0001D76F000E5B
:1001A800D86FD16BD26B390193970DD0000E1B1805
:1001B80002E1000E1A18CAE0000E1B1802E1030E35
:1001C8001A18DEE0F2D7390193AF17D0A3AF15D0D4
:1001D8003C0EB76EB00EB66E1C4A1D2A000E006E9D
:1001E8001D50005C02E11C50090806E2010E446E35
:1001F800000E456E939F938FA39F94A125D0A4A131
:1002080023D0240E3D01EA6F010E465C006E000EFD
:100218004758016E00C046F001C047F0800E4718ED
:10022800006E800E005C02E1010E465C07E2B290AF
:1002380039019491010E1E6E000E1F6E39013C0E9D
:10024800B16EB00EB06EA49117C000F016C001F0E8
:1002580015C002F0600063F0E1FF600067F0E2FFA4
:02026800110083
:0C026A00000E3D01F9BF010E006E1200F5
:0C027600000E3D01E1BF010E006E120001
:04028200F9DF12008E
:04028600F1DF120092
:10028A00FBDF005202E10000FBD767007BFCD2FDD6
:02029A00120050
:10029C00F4DF005202E10000FBD767007BFCEAFDB3
:0202AC0012003E
:0A02AE00670075FC1EFFF3DF12006D
:0A02B800670075FC1EFFEEDF120068
:0A02C200670075FC1EFFE0DF12006C
:0A02CC00670075FC1EFFDBDF120067
:0E02D600026A016A006A086A036A000E1200DA
:1002E4000B820BAE7CEF01F00368026801680068C2
:0802F4000A360232FF0E12006F
:1002FC000B840BAE89EF01F0010E036E026A016AEA
:0A030C00006A0A360232FF0E1200EA
:0E031600550E3A01BF6FAA0EBF6FBF911200C5
:080324000AAE029E000E120059
:10032C00D250026ED29E0500FF6A0150FE6E005044
:08033C00FD6E02BED28E12001C
:0E034400550E3A01BF6FAA0EBF6FBF811200A7
:100352000CB0EBEF01F00CA291EF02F00E6A000E6E
:10036200026402EF02F0F00E0214D8A4CDEF01F005
:10037200023A01380F0B02260138F00B016E0038E9
:100382000F0B01260038F00B006E08380F0B002609
:100392000838F00B086E0E84D89002BEE6EF01F02A
:1003A20008360036013602360E2A02BEE6EF01F0AA
:1003B20008360036013602360E2A02BEE6EF01F09A
:1003C20008360036013602360E2A0E50036487EFD5
:1003D20002F0035E0BBC08AE8CEF02F0D880800EF8
:1003E20008640030000E002201220222D8A08CEF05
:1003F20002F0023201320032034A91EF02F08CEF36
:1004020002F001C002F000C001F008C000F0086A6A
:10041200000E0E86026439EF02F0F00E0214D8A428
:1004220021EF02F0023A01380F0B02260138F00BDD
:10043200016E00380F0B01260038F00B006E0E849F
:10044200D89002BEE6EF01F00036013602360E2ADF
:1004520002BEE6EF01F00036013602360E2A02BE77
:10046200E6EF01F00036013602360E2AE6EF01F021
:1004720001C002F000C001F0006A000E0E960E8864
:10048200026466EF02F0F00E0214D8A451EF02F0FB
:10049200023A01380F0B02260138F00B016E0E846E
:1004A200D89002BEE6EF01F0013602360E2A02BEF5
:1004B200E6EF01F0013602360E2A02BEE6EF01F047
:1004C200013602360E2AE6EF01F001C002F0016A9F
:1004D200000E0E86026496EF02F0F00E0214D8A40B
:1004E20075EF02F0023A0E84D89002BEE6EF01F0F8
:1004F20002360E2A02BEE6EF01F002360E2A02BED4
:10050200E6EF01F002360E2AE6EF01F0010E0C6E64
:10051200F4DE99EF02F0020E0C6E03DF99EF02F0A7
:10052200040E0C6EDEDE99EF02F0080E0C6ED2DEC7
:020532001200B5
:1005340067007BFBE1FF67007FFBE2FF670067FC6E
:10054400E6FF670070FB00F0670074FB01F0ECDE6F
:02055400120093
:100556001F011951170802E2006A0ED31A51000A48
:10056600D8A4B1D01C5301E0D3DE60D067006FFC85
:1005760000FAA5D067006FFC01FAA1D067006FFCF6
:1005860002FA9DD067006FFC03FA99D067006FFCF2
:1005960004FA95D067006FFC05FA91D067006FFCEE
:1005A60006FA8DD067006FFC07FA89D067006FFCEA
:1005B60008FA85D067006FFC09FA81D067006FFCE6
:1005C6000AFA7DD067006FFC0BFA79D067006FFCE2
:1005D6000CFA75D067006FFC0DFA71D067006FFCDE
:1005E6000EFA6DD067006FFC0FFA69D067006FFCDA
:1005F60010FA65D067006FFC11FA61D067006FFCD6
:1006060012FA5DD067006FFC13FA59D067006FFCD1
:1006160014FA55D067006FFC15FA51D067006FFCCD
:1006260016FA4DD067006FFC17FA49D01F01195111
:10063600000A9CE01951010A9DE01951020A9EE048
:100646001951030A9FE01951040AA0E01951050A3D
:10065600A1E01951060AA2E01951070AA3E01951AF
:10066600080AA4E01951090AA5E019510A0AA6E0E8
:1006760019510B0AA7E019510C0AA8E019510D0AE5
:10068600A9E019510E0AAAE019510F0AABE0195157
:10069600100AACE01951110AADE01951120AAEE088
:1006A6001951130AAFE01951140AB0E01951150A8D
:1006B600B1E01951160AB2E01951170AB3E01F0149
:1006C6001C5301E03CDE1F011A51010AD8A451D186
:1006D6001C5301E01DDEA4D0670067FCC0FA45D1BB
:1006E600670067FCC1FA41D1670067FCC2FA3DD1D9
:1006F600670067FCC3FA39D1670067FCC4FA35D1D5
:10070600670067FCC5FA31D1670067FCC6FA2DD1D0
:10071600670067FCC7FA29D1670067FCC8FA25D1CC
:10072600670067FCC9FA21D1670067FCCAFA1DD1C8
:10073600670067FCCBFA19D1670067FCCCFA15D1C4
:10074600670067FCCDFA11D1670067FCCEFA0DD1C0
:10075600670067FCCFFA09D1670067FCD0FA05D1BC
:10076600670067FCD1FA01D1670067FCD2FAFDD0B9
:10077600670067FCD3FAF9D0670067FCD4FAF5D0B6
:10078600670067FCD5FAF1D0670067FCD6FAEDD0B2
:10079600670067FCD7FAE9D0670067FCD8FAE5D0AE
:1007A600670067FCD9FAE1D0670067FCDAFADDD0AA
:1007B600670067FCDBFAD9D0670067FCDCFAD5D0A6
:1007C600670067FCDDFAD1D0670067FCDEFACDD0A2
:1007D600670067FCDFFAC9D0670067FCE0FAC5D09E
:1007E600670067FCE1FAC1D0670067FCE2FABDD09A
:1007F600670067FCE3FAB9D0670067FCE4FAB5D096
:10080600670067FCE5FAB1D0670067FCE6FAADD091
:10081600670067FCE8FAA9D0670067FCE9FAA5D08B
:100826001F011B51000AD8B457D71B51010AD8B46F
:1008360057D71B51020AD8B457D71B51030AD8B44D
:1008460057D71B51040AD8B457D71B51050AD8B439
:1008560057D71B51060AD8B457D71B51070AD8B425
:1008660057D71B51080AD8B457D71B51090AD8B411
:1008760057D71B510A0AD8B457D71B510B0AD8B4FD
:1008860057D71B510C0AD8B457D71B510D0AD8B4E9
:1008960057D71B510E0AD8B457D71B510F0AD8B4D5
:1008A60057D71B51100AD8B457D71B51110AD8B4C1
:1008B60057D71B51120AD8B457D71B51130AD8B4AD
:1008C60057D71B51140AD8B457D71B51150AD8B499
:1008D60057D71B51160AD8B457D71B51170AD8B485
:1008E60057D71B51180AD8B457D71B51190AD8B471
:1008F60057D71B511A0AD8B457D71B511B0AD8B45D
:1009060057D71B511C0AD8B457D71B511D0AD8B448
:1009160057D71B511E0AD8B457D71B511F0AD8B434
:1009260057D71B51200AD8B457D71B51210AD8B420
:1009360057D71B51220AD8B457D71B51230AD8B40C
:1009460057D71B51240AD8B457D71B51250AD8B4F8
:1009560057D71B51260AD8B457D71B51270AD8B4E4
:1009660057D71B51280AD8B457D71F011C5301E08B
:10097600E6DCA8D01F011AB102D0C29001D0C28015
:10098600F9D01F011AB102D0C29201D0C282F2D0B0
:100996001F011AB102D0C29401D0C284EBD01F014C
:1009A6001AB102D0C29601D0C286E4D01F011AB194
:1009B60002D0C29801D0C288DDD01F011AB102D080
:1009C600C29A01D0C28AD6D01F011AB102D0C29CE7
:1009D60001D0C28CCFD01F011AB102D0C29E01D065
:1009E600C28EC8D01F011AB102D0C39001D0C380F5
:1009F600C1D01F011AB102D0C39201D0C382BAD0AE
:100A06001F011AB102D0C39401D0C384B3D01F0111
:100A16001AB102D0C39601D0C386ACD01F011AB159
:100A260002D0C39801D0C388A5D01F011AB102D045
:100A3600C39A01D0C38A9ED01F011AB102D0C39CAB
:100A460001D0C38C97D01F011AB102D0C39E01D02A
:100A5600C38E90D01F011AB102D0C49001D0C480B9
:100A660089D01F011AB102D0C49201D0C48282D0AB
:100A76001F011AB102D0C49401D0C4847BD01F01D7
:100A86001AB102D0C49601D0C48674D01F011AB11F
:100A960002D0C49801D0C4886DD01F011AB102D00B
:100AA600C49A01D0C48A66D01F011AB102D0C49C70
:100AB60001D0C48C5FD01F011AB102D0C49E01D0F0
:100AC600C48E58D01F011951000AD8B453D71951F2
:100AD600010AD8B456D71951020AD8B459D71951B0
:100AE600030AD8B45CD71951040AD8B45FD7195190
:100AF600050AD8B462D71951060AD8B465D7195170
:100B0600070AD8B468D71951080AD8B46BD719514F
:100B1600090AD8B46ED719510A0AD8B471D719512F
:100B26000B0AD8B474D719510C0AD8B477D719510F
:100B36000D0AD8B47AD719510E0AD8B47DD71951EF
:100B46000F0A81E01951100A85E01951110A89E04E
:100B56001951120A8DE01951130A91E01951140A1C
:100B660095E01951150A99E01951160A9DE0195197
:0A0B7600170AA1E0FF0E006E120046
:080B80000B6A0B86FF0E120048
:100B88000B800BAED0EF05F0026A0AAEFF0E026EC4
:0C0B9800016E006E0A360232FF0E1200E1
:100BA4000C6A0E6A0250D8A4EBEF05F001C002F003
:100BB40000C001F0006A0E860250D8A4EBEF05F0E5
:100BC40001C002F0016A0E960E880250D8B4FDEFFF
:100BD40005F00E50035ED8A4D8A003EF06F0D89019
:100BE40002BE09EF06F0003601360236032EF2EF9C
:100BF40005F003EF06F0010E0C6E6BEC01F00DEF47
:100C040006F0020E0C6E7EEC01F00DEF06F0040E01
:080C14000C6E92EC01F01200DD
:100C1C001F01186B670057FCE9FF67005BFCEAFFDC
:100C2C006F00B9FF17FF1751000A10E067005DFC59
:100C3C0019FF7ADC1F01182B18511525E96E000ECF
:0E0C4C001621EA6E6F00B9FF17FFEDD71200F8
:100C5A00670055FC19FF670059FC1AFF67005DFC25
:0C0C6A001BFF010E1F011C6F71DC12004B
:100C7600025006180E6E086A096A0B6A035007646A
:100C86002EEF07F006500A6E068E028E03500B6E8C
:100C96000750036E000E0B647EEF06F00B50075EE6
:100CA600D8B41FEF07F0070E0764EDEF06F0075EF6
:100CB60000C008F001C000F002C001F0026A074E51
:100CC6001FEF07F00764C2EF06F0075E00C008F0EA
:100CD60001C000F0016A074E1FEF07F00764A0EF9E
:100CE60006F0075E00C008F0006A074E1FEF07F027
:100CF600076487EF06F00AC002F005C001F004C0E1
:100D060000F0086A4BEF08F0030E076492EF06F056
:100D1600075E08380F0B086E074E1FEF07F0D890D6
:100D26000832074E1FEF07F0D8900832074E1FEF24
:100D360007F0D89008321FEF07F0030E0764B1EFF3
:100D460006F0075E08380F0B086E0038F00B082611
:100D560000380F0B006E074E1FEF07F0D8900032D9
:100D66000832074E1FEF07F0D89000320832074EC0
:100D76001FEF07F0D890003208321FEF07F0030E7E
:100D86000764D9EF06F0075E08380F0B086E0038C7
:100D9600F00B082600380F0B006E0138F00B00260A
:100DA60001380F0B016E074E1FEF07F0D890013286
:100DB60000320832074E1FEF07F0D890013200329A
:100DC6000832074E1FEF07F0D89001320032083282
:100DD6001FEF07F0030E07640AEF07F0075E0838F7
:100DE6000F0B086E0038F00B082600380F0B006E4C
:100DF6000138F00B002601380F0B016E0238F00B9C
:100E0600012602380F0B026E074E1FEF07F0D8902F
:100E16000232013200320832074E1FEF07F0D89037
:100E26000232013200320832074E1FEF07F0D89027
:100E36000232013200320832096A000E0EAE13EF9A
:100E460008F0081E001E011E021E082A00220122AA
:100E5600022213EF08F00750D8A434EF07F04BEF47
:100E660008F0096A02C00AF0028E068E0750035C7B
:100E7600076ED8B406EF08F0070E0764D4EF07F044
:100E8600075E0450096E0550046E0650056E066A2C
:100E9600074E06EF08F0070E0764A9EF07F0075E96
:100EA6000450096E0550046E056A074E06EF08F0F9
:100EB600070E076487EF07F0075E0450096E046AA1
:100EC600074E06EF08F0070E07646EEF07F00AC03C
:100ED60002F04BEF08F0030E076479EF07F0075EA8
:100EE60009380F0B096E074E06EF08F0D890093245
:100EF600074E06EF08F0D8900932074E06EF08F0C5
:100F0600D890093206EF08F0030E076498EF07F051
:100F1600075E09380F0B096E0438F00B09260438F2
:100F26000F0B046E074E06EF08F0D8900432093214
:100F3600074E06EF08F0D89004320932074E06EF46
:100F460008F0D8900432093206EF08F0030E076461
:100F5600C0EF07F0075E09380F0B096E0438F00B77
:100F6600092604380F0B046E0538F00B04260538E5
:100F76000F0B056E074E06EF08F0D89005320432C7
:100F86000932074E06EF08F0D890053204320932CE
:100F9600074E06EF08F0D89005320432093206EF04
:100FA60008F0030E0764F1EF07F0075E09380F0B30
:100FB600096E0438F00B092604380F0B046E053849
:100FC600F00B042605380F0B056E0638F00B0526C8
:100FD60006380F0B066E074E06EF08F0D89006325D
:100FE600053204320932074E06EF08F0D890063271
:100FF600053204320932074E06EF08F0D890063261
:10100600053204320932086A000E0EAE13EF08F0FC
:10101600091E041E051E061E092A04220522062292
:1010260009500826045000220550012206500222CB
:101036000EBE2AEF08F0D8A039EF08F002320132CE
:1010460000320832033E39EF08F045EF08F0D8B019
:101056003FEF08F0000E081E001E011E021E082AA1
:101066000022012202220A7E3FEF08F0010E0C6EDA
:10107600A9EC01F04DEF08F0020E0C6EA9EC01F0A0
:101086004DEF08F0040E0C6E72EC01F04DEF08F017
:06109600000E0C6E1200BA
:10109C00670024FC00F01F010907005232E06700D2
:1010AC0017FCE9FF67001BFCEAFFEE50000A10E09A
:1010BC00670017FCE9FF67001BFCEAFF67001FFCD9
:1010CC00D9FF670023FCDAFFEE50DE1801E113D0E4
:1010DC00670017FCE9FF67001BFCEAFF67001FFCB9
:1010EC00D9FF670023FCDAFFDE50EE5C006E016A6C
:1010FC00000E015A08D01F01054B062B074B082B7D
:08110C00C7D7006A016A120056
:101114000D0E1F011D6F57EC01F00A0E1F011D6F0C
:0611240057EC01F012007F
:06112A00067EA4DD1200A8
:101130000B6A0350D8B4DEEF08F002500A6E028E3C
:101140008E0E035E03AEE2EF08F0036C080E035C44
:10115000D8A0BDEF08F0036E013602C001F0026AAC
:10116000080E035CD8A0BDEF08F0036E0136016ADB
:101170000350D8A4D890C7EF08F00350D8B4C7EFF5
:1011800008F0D89002320132032EC1EF08F00BBCF8
:1011900001A0D4EF08F0D8A0D4EF08F0012AD8B409
:1011A000022A02BEF1EF08F00AAEF6EF08F0021EC6
:1011B000011E012AD8B4022AF6EF08F0026A016A79
:1011C000F6EF08F00B800BAEFAEF08F0026A0AAEF9
:1011D000FAEF08F0FF0E026E016E0A360232FAEFE5
:1011E00008F0010E0C6ED0DCFCEF08F0000E0C6E67
:1011F000FCEF08F0FF0E0C6E0150006E0250016E05
:021200001200DA
:0C1202006F00A0F701F001C000F0120026
:10120E00670014FC00F00032009E0032009E003297
:10121E00009E0032009E150E0024F66E390EF76EFB
:10122E00000EF722000EF86E000EF82209006F0075
:10123E00D4FF00F067001BFCE1FF67001FFCE2FF1C
:10124E00600003F0E6FF010E1F010625E16E000EA1
:10125E000721E26E0F0E0515006E150E0024F66EB8
:10126E00390EF76E000EF722000EF86E000EF82201
:10127E0009006F00D4FF00F0600003F0E6FF020EDD
:0E128E000625E16E000E0721E26EE66A1200F0
:10129C00670017FCE9FF67001BFCEAFFEE501F011B
:1012AC00071907E1670014FC00F0670018FC01F057
:1012BC0015D0670014FC00F0670018FC01F0054B1A
:1012CC00062B600003F0E9FF600007F0EAFF6F00F7
:0E12DC00B8FF00F00052DCE1006A016A120067
:1012EA00086A096A000E07620364FDEF09F00250FA
:1012FA0006180A6E075003267E0ED8A08BEF09F057
:10130A00035ED8B002EF0AF08FEF09F0035ED8A0AF
:10131A0007EF0AF0028E068E02C00EF001C00BF033
:10132A0000C00DF0005004026F00D0FF0CF0015015
:10133A0005026F00D0FF00F06F00CCFF08F0040236
:10134A00F3500C26F4500822000E00220D5005021C
:10135A00F3500C26F4500822000E00220250040218
:10136A00F3500826F450002202500502016A000ECA
:10137A000122F3500026F45001220D500602F350C8
:10138A000826F4500022026A000E012202220B50A3
:10139A000602F3500026F4500122000E02220E50DB
:1013AA000602F3500126F450022202BEE5EF09F0CC
:1013BA0008360036013602360306D8B407EF0AF0BB
:1013CA00F8EF09F0D880800E08640030000E002281
:1013DA0001220222D8A0F8EF09F0023201320032CB
:1013EA00034A02EF0AF00AAE029E000E0AEF0AF062
:1013FA00010E6BEC01F00AEF0AF0020E72EC01F03A
:0C140A000AEF0AF0040E7EEC01F0120064
:101416001F0105510308D8A0056B06510308D8A083
:10142600066BF00E3D01F2171F0105513D01F21347
:10143600300EF213670018FC00F0003600900036FC
:10144600009000360090003600900050F413F38FA1
:02145600120082
:10145800670015FCD8FE670019FCD9FE67001DFC63
:10146800DAFE670021FCDBFE670025FCDCFE670076
:1014780029FCDDFE67002DFCDEFE670031FCDFFE87
:10148800670035FCD4FE670039FCD5FE67003DFCDB
:10149800D6FE670041FCD7FE670045FCCEFE67001C
:1014A80049FCCFFE67004DFCD0FE670051FCD1FE21
:0214B800120020
:1014BA000A6A0350D8A40A800750D8A40A820A509C
:1014CA00D8B4C0EF0AF0030AD8B479EF0AF00AB028
:1014DA0074EF0AF006AEBEEF0AF0BCEF0AF002AEF5
:1014EA00BCEF0AF0BEEF0AF00250800B0A6E029EB1
:1014FA000650800B069E0A18D8B48AEF0AF00A50E2
:10150A00D8B4BCEF0AF0BEEF0AF00750035CD8B4B7
:10151A0094EF0AF0D8A0B0EF0AF0B6EF0AF006503E
:10152A00025CD8B49EEF0AF0D8A0B0EF0AF0B6EF8A
:10153A000AF00550015CD8B4A8EF0AF0D8A0B0EFC1
:10154A000AF0B6EF0AF00450005CD8B4C0EF0AF013
:10155A00D8B0B6EF0AF00A52D8B4BEEF0AF0BCEF20
:10156A000AF00A52D8B4BCEF0AF0BEEF0AF0D880EB
:0E157A001200D8901200D880D88412001200FF
:101588000B6A0A6A096A005004026F00D0FF09F06A
:101598006F00CCFF08F0015005026F00D0FF0BF080
:1015A8006F00CCFF0AF000500502F3500926F450F2
:1015B8000A22E86A0B2201500402F3500926F4506B
:1015C8000A22E86A0B2208C000F009C001F00AC02C
:0815D80002F00BC003F0120049
:0A15E000750E0D6E0D2EFED71200E1
:1015EA000450000A12E10550000A0FE10650000AF1
:1015FA000CE10750000A09E1FF0E006EFF0E016EB2
:10160A007F0E026EFF0E036EA8D0086A096A0750A1
:10161A00D8B4A0EF0BF00350D8B4A5EF0BF00250EA
:10162A0006180A6E028E068E0E6A02C008F001C003
:10163A000CF000C00DF004500D5E0550D8A0053C1A
:10164A000C5E0650D8A0063C085E086A0C6A0D6A51
:10165A00D8A037EF0BF0D8900232013200320832AC
:10166A00010E0E6E0750035ED8A044EF0BF07E0EFB
:10167A000E240326D8B0AAEF0BF04AEF0BF07E0E29
:10168A000E240326D8A0AFEF0BF0180E0B6E0D3602
:10169A000C3608360036013602360E360450005E25
:1016AA000550D8A0053C015E0650D8A0063C025E53
:1016BA0006340E120EA065EF0BF00D8070EF0BF0E2
:1016CA00045000260550D8B0053C01260650D8B073
:1016DA00062802260D900B2E4CEF0BF096EF0BF01E
:1016EA00D8900036013602360E360450005E055098
:1016FA00D8A0053C015E0650D8A0063C025E06341E
:10170A000E10010B0D26D8B00C2AD8B4082AD8A47A
:10171A0096EF0BF008320C320D32032AD8B4AAEF36
:10172A000BF00AAE089E0850026E0C50016E0D5066
:10173A00006EB2EF0BF0010EC0EC05F0B2EF0BF049
:10174A00020E6BEC01F0B2EF0BF0040E72EC01F03A
:0C175A00B2EF0BF0080E7EEC01F0120064
:10176600670015FC15FF670019FC16FF0EEC06F066
:0217760012005F
:10177800670014FC02F0670018FC03F002C000F0D8
:1017880003C001F0024A032A600003F0E9FF600089
:1017980007F0EAFFEE5201E0F1D71F010551025CA4
:1017A800006E06510358016E010E005E000E015ACC
:0217B80012001D
:1017BA0000C008F00150006E016A026A036A0B6AEF
:1017CA000C6A016A026A036A960E036E0A6A00AE1E
:1017DA00F5EF0BF0081E001E082AD8B4002A0A8E5C
:1017EA0000C001F008C000F0086A026AD2EC05F0F5
:0217FA001200DB
:1017FC00FC0E3F015E175E81010EAE6E7C6A7D6A47
:02180C001200C8
:10180E00160E1F01156F166B130E176F2DEC06F0CB
:10181E00170E1F01156F010E166F250E176F2DEC8B
:04182E0006F01200AE
:10183200086A096A100E0C6E013408360936045023
:10184200085E0550D8A0053C095ED8B007D0045008
:1018520008260550D8B0053C0926D8900036013636
:061862000C2EEAD7120073
:10186800000E1E01ED1902E1000EEC1948E06700B8
:10187800B3FBE9FF6700B7FBEAFFEE5240E0670001
:10188800B9FB05FF6700BDFB06FF72DF600001F0D2
:1018980009FF6700B1FB05FF6700B5FB06FF67009E
:1018A800B9FB07FF6700BDFB08FF4EEC08F0000E10
:1018B800011802E1000E001807E16700B0FB00F014
:1018C8006700B4FB01F01DD0010E1E01EC251F01BD
:1018D800056F000E1E01ED211F01066F6700BBFB9F
:1018E800E9FF6700BFFBEAFF6F00B9FF07FFD2DC23
:1018F800600001F0ECFE600005F0EDFEB1D7006A73
:04190800016A12005E
:10190C003901C06BC16BC26BCA6A020E3A01406FDF
:10191C00A30EC26E439DBA96416B506BCB6A010EFF
:10192C00C36EFF0E516F3E01BC6BB86BC3823901A5
:10193C00C06BCC6A3A01606B800EC46EC49ABC9AC0
:10194C00C296BA963E01C16BC18FC183C1913A0157
:04195C00636B1200A7
:101960006700B3FBE9FF6700B7FBEAFFEE50000832
:101970000FE26700B3FBE9FF6700B7FBEAFF6F0008
:10198000B9FF1DFF57EC01F01E01EC4BED2BE8D722
:02199000120043
:101992006700B3FBF6FF6700B7FBF7FF6700BBFB0F
:1019A200F8FF09006F00D4FF01F00150000816E2B1
:1019B2006700B3FBF6FF6700B7FBF7FF6700BBFBEF
:1019C200F8FF09006F00D5FF1DFF57EC01F0010E73
:0E19D2001E01EC27000EED23EE23DAD71200E3
:1019E0006700BBFBF6FF6700BFFBF7FF6700C3FBA9
:1019F000F8FF09006F00D4FF00F000521FE06700FD
:101A0000BBFBF6FF6700BFFBF7FF6700C3FBF8FFF8
:101A100009006F00D4FF00F06700B3FBE1FF67002F
:101A2000B7FBE2FF600003F0E6FF1E01EC4BED2B7D
:101A3000010EEE27000EEF23F023D2D76700B3FB91
:0C1A4000E1FF6700B7FBE2FFE66A12005E
:101A4C006700B8FB04F06700BCFB05F06700B0FB57
:101A5C0002F06700B4FB03F06700C0FB00F0670006
:101A6C00C4FB01F0010E1E01F05F000EF15B005093
:101A7C00011014E0600013F0E9FF600017F0EAFFBA
:101A8C0060000BF0E1FF60000FF0E2FF6F00BBFFA6
:101A9C00E6FF024A032A044A052ADED76700B0FB98
:0A1AAC0000F06700B4FB01F0120027
:061AB60001EC09F0120032
:101ABC00A8DEB60E1F01056F1A0E066F000E076F1B
:101ACC00000E086FAE0E096F020E0A6F1D0E0B6F23
:101ADC001F0E0C6FFF0E0D6FFF0E0E6F000E0F6FB3
:101AEC00000E106F860E116F020E126F000E136F28
:0E1AFC00000E146FABDC056B066B87DC12006E
:101B0A0009006F00D7FFE6FF0006FAE10106F8E1D7
:021B1A001200B7
:101B1C000050086E0150006E016A026A036A0B6A7B
:101B2C000C6A960E036E0A6A00C001F008C000F041
:0A1B3C00086A026AD2EC05F01200FC
:101B4600BC8A0001D16BD26B000ED25D02E17F0E22
:101B5600D15D18E2510ED125E16E000ED221E26E62
:101B66006F0087FFE1FF6F008BFFE2FFE66A010E61
:101B7600D125006E000ED221016E00C0D1F001C049
:101B8600D2F0E2D7516AD16BD26BD36BD46BD76BE1
:101B9600D86B3D01F289F96BFA6B486A3901938774
:041BA600BC9A1200D3
:101BAA00120E1F01156F166B090E176F2DEC06F03A
:041BBA0020DE120017
:101BBE001E01F251000805E3070EF36F000EF46FDD
:101BCE0014D0F251160805E2170EF56F000EF66FDF
:101BDE0006D0F251010FF56FF66B000EF62367007B
:101BEE00D5FBF3FE6700D9FBF4FE6700CDFBFDFECF
:101BFE006700D1FBFEFEF76BF86B046A056A066A96
:101C0E00076A6700B0FB00F06700B4FB01F06700E5
:101C1E00B8FB02F06700BCFB03F048DC010ED8B045
:101C2E00000E006E00520BE06700C3FBE1FF670081
:101C3E00C7FBE2FF2D0EE66EF04BF12BEE7F670039
:101C4E00B0FB04F06700B4FB05F06700B8FB06F0CC
:101C5E006700BCFB07F0006A016A026A036A26DCB1
:101C6E00010ED8B0000E006E005242E0000E046E5F
:101C7E00000E056E000E066E7F0E076E6700B0FB3F
:101C8E0000F06700B4FB01F06700B8FB02F06700DC
:101C9E00BCFB03F00BDC010ED8B0000E006E005240
:101CAE0027E06700B0FB00F06700B4FB01F06700AF
:101CBE00B8FB02F06700BCFB03F0000E046E000ED2
:101CCE00056E200E066E820E076E75EC09F0600032
:101CDE0001F0ECFE600005F0EDFE600009F0EEFE96
:101CEE0060000DF0EFFE010EF75F000EF85BBED741
:101CFE00000E046E000E056E200E066E820E076E2E
:101D0E006700B0FB00F06700B4FB01F06700B8FBA2
:101D1E0002F06700BCFB03F05DEC0AF0000ED8B0D9
:101D2E00010E006E005225E0000E046E000E056ED0
:101D3E00200E066E820E076E6700B0FB00F0670085
:101D4E00B4FB01F06700B8FB02F06700BCFB03F0C8
:101D5E0045DC600001F0ECFE600005F0EDFE600079
:101D6E0009F0EEFE60000DF0EFFE1E01F74BF82BB2
:101D7E00BFD7F751FD27F851FE23010EF96F000E64
:101D8E00FA6F000E1F01016F000E026F000E036F3F
:101D9E007F0E046F800E1E01FA19006E800EFE1962
:101DAE00005C02E1FD51F95D25E2000E046E000EAD
:101DBE00056E200E066E820E076E670004FC00F0A4
:101DCE00670008FC01F067000CFC02F0670010FCD5
:101DDE0003F004DC600001F001FF600005F002FF7B
:101DEE00600009F003FF60000DF004FF1E01F94BC7
:101DFE00FA2BD0D7000E046E000E056E000E066E86
:101E0E00800E076E670004FC00F0670008FC01F00E
:101E1E0067000CFC02F0670010FC03F0F5EC0AF012
:101E2E006700B0FB04F06700B4FB05F06700B8FB79
:101E3E0006F06700BCFB07F03BEC06F0600001F01B
:101E4E00ECFE600005F0EDFE600009F0EEFE6000B5
:101E5E000DF0EFFE000E046E000E056E200E066EE7
:101E6E00820E076E5DEC0AF0000ED8B0010E006E09
:101E7E0000520BE0000E1E01EC6F000EED6F000E17
:101E8E00EE6F7F0EEF6FF74BF82B1E01800EF819D9
:101E9E00006E800E005C02E1000EF75D3EE2670010
:101EAE00C3FBE1FF6700C7FBE2FF300EE66EF04BAF
:101EBE00F12B6700C3FBE1FF6700C7FBE2FF2E0EAD
:101ECE00E66EF04BF12B800EFE19006E800E005C5C
:101EDE0002E1000EFD5D04E2FD51F75FFE51F85B7D
:101EEE00FF0EF96FFF0EFA6F800EF819006E800E5E
:101EFE00FA19005C02E1F951F75D0FE26700C3FBCE
:101F0E00E1FF6700C7FBE2FF300EE66EF04BF12BF0
:101F1E00010EF95F000EFA5BE7D7F96BFA6B800ED4
:101F2E00FA19006E800EFE19005C02E1FD51F95D9A
:101F3E00D8B07FD06700B0FB00F06700B4FB01F0B3
:101F4E006700B8FB02F06700BCFB03F098EC08F0EA
:101F5E00600001F0FBFE600005F0FCFE300E002676
:101F6E006700C3FBE1FF6700C7FBE2FF600003F001
:101F7E00E6FFF04BF12BFA51F81902E1F751F9197E
:101F8E000AE16700C3FBE1FF6700C7FBE2FF2E0E0D
:101F9E00E66EF04BF12B6700ECFB00F06700F0FBF8
:101FAE0001F004DC600001F001FF600005F002FFAB
:101FBE00600009F003FF60000DF004FF00C004F0A4
:101FCE0001C005F002C006F003C007F06700B0FBC9
:101FDE0000F06700B4FB01F06700B8FB02F0670089
:101FEE00BCFB03F095EC08F0600001F0ECFE600025
:101FFE0005F0EDFE600009F0EEFE60000DF0EFFE64
:10200E00000E046E000E056E200E066E820E076E1A
:10201E0075EC09F0600001F0ECFE600005F0EDFEDD
:10202E00600009F0EEFE60000DF0EFFEF94BFA2BAA
:10203E0076D76700C3FBE1FF6700C7FBE2FFE66AE6
:02204E0012007E
:082050007E9EF00E7E161200C8
:102058001E01F06B050EF05D0AE2F051EE25E16E0F
:10206800000EEF21E26E200EE66EF02BF3D7F05152
:10207800EE25E16E000EEF21E26EE66AF007F05100
:10208800EE25F16F000EEF21F26F0A0E046E000EBE
:10209800056E6700B0FB00F06700B4FB01F019ECB7
:1020A8000CF008C000F009C001F0300E00266700EF
:1020B800C7FBE1FF6700CBFBE2FF600003F0E6FF30
:1020C8000A0E046E000E056E6700B0FB00F0670094
:1020D800B4FB01F019EC0CF0600001F0ECFE6000BC
:1020E80005F0EDFE000E011802E1000E001801E1F6
:0820F80002D0F007C4D712006A
:0A210000AC8E7E8E0C0E7E121200D3
:10210A001E01F46BF56B6700B9FBF6FE6700BDFBB9
:10211A00F7FEF733F633F79FF733F633F79FF733C4
:10212A00F633F79FF733F633F79F000EEF5D02E1C0
:10213A00100EEE5D35E2200E1F011D6F57EC01F007
:10214A001E01F06BF16BEF51F15D02E1EE51F05DB2
:10215A0024E2F051EC25E96EF151ED21EA6E6F00AF
:10216A00A7FFE9FF6F00ABFFEAFF6F00B9FF05FFAA
:10217A00FA0E1F01066F1E0E076F07EC09F0FA0E22
:10218A00056F1E0E066FB3EC0BF02E0E1D6F57EC8B
:10219A0001F01E01F04BF12BD6D78AEC08F0C3D020
:1021AA001E01F26BF36BF751F35D02E1F651F25D3A
:1021BA0054E2200E1F011D6F57EC01F01E01F06B57
:1021CA00F16B000EF15D02E1100EF05D40E2670076
:1021DA00C8FB00F06700CCFB01F000360090013626
:1021EA000036009001360036009001360036009025
:1021FA000136F0510026F1510122600001F0F4FE8F
:10220A00600005F0F5FE0050EC25E96E0150ED2165
:10221A00EA6E6F00A7FFE9FF6F00ABFFEAFF6F00EE
:10222A00B9FF05FFFA0E1F01066F1E0E076F07ECB6
:10223A0009F0FA0E056F1E0E066FB3EC0BF02E0EA8
:10224A001D6F57EC01F01E01F04BF12BBAD78AEC47
:10225A0008F01E01F24BF32BA6D76700D8FB00F05B
:10226A006700DCFB01F00036009001360036009072
:10227A0001360036009001360036009001366000C3
:10228A0001F0F4FE600005F0F5FE0050EE5D026E0E
:10229A000150EF59036E600009F0F8FE60000DF07E
:1022AA00F9FE000E006E0350005C02E102500008C5
:1022BA003AE2200E1F011D6F57EC01F01E01F26B6E
:1022CA00F36BF951F35D02E1F851F25D2AE2F45140
:1022DA00EC25006EF551ED21016EF2510024E96EF4
:1022EA00F3510120EA6E6F00A7FFE9FF6F00ABFF11
:1022FA00EAFF6F00B9FF05FFFA0E1F01066F1E0EF7
:10230A00076F07EC09F0FA0E056F1E0E066FB3ECA5
:10231A000BF02E0E1D6F57EC01F01E01F24BF32B42
:0C232A00D0D78AEC08F08AEC08F0120012
:10233600AA0E1E01E86F230EE96FEC0EEA6F1E0E61
:10234600EB6F3E01F86BF96BFA6BFB6BEC0EFD174E
:10235600130E1E01EC15006E00503E01FD13C00E5B
:102366001E01EC15006E17E0C00EEC15026E060E8F
:10237600016E02C000F0015004E00032009EFF0F23
:10238600FBD7600003F0C1FE3E01C18FC1BD02D084
:102396000000FCD703D03E01FC0EC117F889F88572
:0423A600F88F12009A
:1023AA003F0E1E01EC153E01F16FF0EC0AF0F881C8
:1023BA000000F8A101D0FDD76F00BCFB00F06F0050
:0623CA00C0FB01F012004F
:1023D000AB50010F006E016A000E01226700B0FBD6
:1023E00004F06700B4FB05F0C4EC0AF0060E046EBE
:1023F00000C002F001C003F0045005E003320232D5
:10240000039EFF0FFAD760000BF07CFF60000FF017
:042410007DFF12003A
:10241400F5EC1CF0600E3901D96FDA51D91902E0DC
:10242400DB6BFBD7DD6B080EDF6FDE6BD98DD98BD1
:10243400D999D997D995D993D9916E0070F720F08D
:1024440086EC0CF00001DD951E6A1F6A1C6A1D6A89
:10245400DB6BDC6B000EDC5D02E1080EDB5D11E280
:10246400BA78150E0B6E4B0E0C6EBE0E0D6E0D2E45
:10247400FED70C2EFCD70B2EFAD70000DB4BDC2B3F
:10248400E9D7DB6BDC6B000EDC5D02E1500EDB5D3B
:1024940010E2DE0EDB25E16E000EDC21E26E6F0041
:1024A40087FFE1FF6F008BFFE2FFE66ADB4BDC2B6B
:1024B400EAD7BA98DB6BDC6B1D0EDC5D02E14C0ED7
:1024C400DB5D10E2820EDB25E16E010EDC21E26EA3
:1024D4006F0087FFE1FF6F008BFFE2FFE66ADB4BD3
:1024E400DC2BEAD78BEC01F0156B090E126F130E7F
:1024F400166F170EE56FA2EC01F0400E3D01F56F6B
:10250400030EF66FF28F5EEC0DF0B60E1F01056F31
:102514001A0E066F000E076F000E086FAE0E096FDD
:10252400020E0A6F1D0E0B6F1F0E0C6FFF0E0D6F48
:10253400FF0E0E6F000E0F6F000E106F860E116FE0
:10254400020E126F000E136F000E146F2CEC0AF0C3
:10255400520E0B6E2B0E0C6E000E0D6E0D2EFED752
:102564000C2EFCD70B2EFAD700003D01F491F49306
:10257400F48F0C0E1F011D6F57EC01F0A60E1E0107
:10258400EC6F380EED6F000EEE6FC9EC0CF000012D
:10259400DB6BDC6B000EDC5D02E10A0EDB5D25E229
:1025A400030E006E000E016EDBC004F0DCC005F00B
:1025B400C4EC0AF0210E0024E96E000E0120EA6E3C
:1025C4006F00A7FFE9FF6F00ABFFEAFF6F00B9FFE1
:1025D400ECFE6F00B9FFEDFE6F00B9FFEEFEC9EC33
:1025E4000CF00001DB4BDC2BD5D739015B918AEC75
:1025F40008F02E0E0101806F010E816FDC0E1E01AA
:10260400EC6F340EED6F000EEE6FC9EC0CF01E0192
:10261400EC6B8FDEBA980D0E1E01EC6F360EED6F6B
:10262400000EEE6FC9EC0CF001017E6B7F6BED0EBA
:102634001E01EC6F360EED6F000EEE6FC9EC0CF060
:10264400800E01017E6F000E7F6F300EAC12B50E4E
:10265400AB6ED5EC0DF0BA8651DD6000F9F5ECFEF9
:102664006000FDF5EDFEB2DEBA960001D96BDA6BBF
:102674004B6A4C6A4D6A4E6AD76AD66A080ED56EA2
:10268400D28E1A6A1B6A496A4A6A100E4F6E000E8D
:10269400506E010ED56F000ED66F39019491FF0E66
:1026A400426EFF0E436EBC8AE7EF19F0FF0E426ED6
:1026B400FF0E436E010E1E01EC6F75DE00C04DF07F
:1026C40001C04EF000504B2601504C220001D94B62
:1026D400DA2B000E006EDA51005C02E1D9510708D2
:1026E400D8B082D0660E1E01EC6F390EED6F000E6D
:1026F400EE6FC9EC0CF04BC000F04CC001F001329D
:102704000032019E01320032019E01320032019EEC
:1027140000C04BF001C04CF00001DE6B600001F022
:10272400ECFE600005F0EDFEDE0E1E01EE6F000E05
:10273400EF6F90DCDE0E1F01056F000E066FB3EC29
:102744000BF0CA0E1E01EC6F390EED6F000EEE6F2A
:10275400C9EC0CF04BC000F04CC001F08EEC0DF055
:10276400000E046E000E056E340E066E7B0E076EB0
:1027740075EC09F0600001F0E2FE600005F0E3FE94
:10278400600009F0E4FE60000DF0E5FE0001DE6B80
:10279400600001F0ECFE600005F0EDFE600009F061
:1027A400EEFE60000DF0EFFEDE0E1E01F06F000E77
:1027B400F16F020EF26FDFEC0DF0DE0E1F01056FFC
:1027C400000E066FB3EC0BF0DD0E1E01EC6F390E3C
:1027D400ED6F000EEE6FC9EC0CF08AEC08F04B6A5A
:1027E4004C6A0001D96BDA6BBA780400496A4A6A08
:1027F400D16BD26BA3EC0DF0520E0B6E2B0E0C6E44
:10280400000E0D6E0D2EFED70C2EFCD70B2EFAD714
:10281400000015EF1AF01ADC420E1E01EC6F390E9F
:10282400ED6F000EEE6FC9EC0CF0510E0001D36F8A
:10283400000ED46F60004DF3ECFE600051F3EDFE2A
:10284400400E1E01EE6F000EEF6F5DDCA50E1E0143
:10285400EC6F390EED6F000EEE6FC9EC0CF0DE0E6E
:102864001E01EC6F000EED6FD80EEE6F390EEF6F98
:10287400000EF06FF0EC0CF0510E1E01EC6F000E28
:10288400ED6FDE0EEE6F000EEF6F34EC0CF000C057
:10289400D3F001C0D4F0000E026E0150025C02E1DC
:1028A40000500008D8B08AD07C0E1E01EC6F390E9F
:1028B400ED6F000EEE6FC9EC0CF0600025F1ECFE3C
:1028C400600029F1EDFEDE0E1E01EE6F000EEF6FCB
:1028D4002CEC10F0DE0EEC6F000EED6FB0EC0CF093
:1028E4008AEC08F0E30E1E01EC6F380EED6F000E5B
:1028F400EE6FC9EC0CF0BB0E1E01EC6F380EED6FE1
:10290400000EEE6FC9EC0CF0050E0001D325E96E44
:10291400000ED421EA6E6F00A7FFE9FF6F00ABFF42
:10292400EAFF6F00B9FFE0FE000E1E01E16F000E2A
:10293400E16F670080FB01F0006A600001F0E0FED7
:10294400600005F0E1FE040E0001D325D96E000EEF
:10295400D421DA6E6F0067FFD9FF6F006BFFDAFFD7
:10296400DE500026000E0122080E0026000E012271
:10297400600001F0E0FE600005F0E1FE00C042F0FE
:1029840001C043F0600001F0ECFE600005F0EDFED4
:10299400DE0E1E01EE6F000EEF6F2CEC10F0DE0E5B
:1029A400EC6F000EED6FB0EC0CF09B0E1E01EC6FA3
:1029B400390EED6F000EEE6FC9EC0CF0DE0E1E0149
:1029C400EC6F000EED6FB80EEE6F390EEF6F000E68
:1029D400F06FF0EC0CF0590E1E01EC6F000EED6F71
:1029E400DE0EEE6F000EEF6F34EC0CF000C0D3F08F
:1029F40001C0D4F0000E026E0150025C02E10050EE
:102A040000081BE2610E1E01EC6F380EED6F000E24
:102A1400EE6FC9EC0CF0090E0B6E1E0E0C6EE40E7C
:102A24000D6E0D2EFED70C2EFCD70B2EFAD7000000
:102A3400020E1A6E000E1B6E2BD0E20E1E01EC6FFE
:102A4400390EED6F000EEE6FC9EC0CF0670099FBC8
:102A5400ECFE67009DFBEDFEDE0E1E01EE6F000E28
:102A6400EF6F2CEC10F0DE0EEC6F000EED6FB0EC9F
:102A74000CF08AEC08F01A6A1B6A496A4A6A990ED1
:102A84001E01EC6F370EED6F000EEE6FC9EC0CF00B
:102A940015EF1AF08AEC08F0510E0001D36F000E06
:102AA400D46F130E1E01EC6F380EED6F000EEE6F37
:102AB400C9EC0CF0250E1E01EC6F390EED6F000E03
:102AC400EE6FC9EC0CF0610E0001D36F000ED46FF1
:102AD400DE0E1E01EC6F000EED6F60004DF3EEFE96
:102AE400600051F3EFFE040EF06F000EF16F26EC60
:102AF4000DF0010E0001D325E96E000ED421EA6E1B
:102B04006F00A7FFE9FF6F00ABFFEAFF6F00B9FF9B
:102B1400E0FE000E1E01E16F000EE16F670080FB16
:102B240001F0006A600001F0E0FE600005F0E1FEE3
:102B340060004FF3D9FF600053F3DAFFDE50002644
:102B4400000E0122600001F0E0FE600005F0E1FEED
:102B5400600001F0ECFE600005F0EDFEDE0EEE6FAD
:102B6400000EEF6F2CEC10F0DE0EEC6F000EED6F2C
:102B7400B0EC0CF08AEC08F0340E1E01EC6F390E48
:102B8400ED6F000EEE6FC9EC0CF0650E0001D36F13
:102B9400000ED46FDE0E1E01EC6F000EED6F6000B0
:102BA4004DF3EEFE600051F3EFFE020EF06F000EE7
:102BB400F16F26EC0DF0010E0001D325E96E000E35
:102BC400D421EA6E6F00A7FFE9FF6F00ABFFEAFFB5
:102BD4006F00B9FFE0FE000E1E01E16F000EE16F11
:102BE400670080FB01F0006A600001F0E0FE600015
:102BF40005F0E1FE60004FF3D9FF600053F3DAFF04
:102C0400DE500026000E0122600001F0E0FE6000AC
:102C140005F0E1FE600001F0ECFE600005F0EDFE61
:102C2400DE0EEE6F000EEF6F2CEC10F0DE0EEC6F8C
:102C3400000EED6FB0EC0CF08AEC08F0F50E1E01FE
:102C4400EC6F380EED6F000EEE6FC9EC0CF0670EF2
:102C54000001D36F000ED46FDE0E1E01EC6F000E68
:102C6400ED6F60004DF3EEFE600051F3EFFE020ED7
:102C7400F06F000EF16F26EC0DF0010E0001D3256C
:102C8400E96E000ED421EA6E6F00A7FFE9FF6F0022
:102C9400ABFFEAFF6F00B9FFE0FE000E1E01E16F1B
:102CA400000EE16F670080FB01F0006A600001F034
:102CB400E0FE600005F0E1FE60004FF3D9FF600024
:102CC40053F3DAFFDE500026000E0122600001F00B
:102CD400E0FE600005F0E1FE600001F0ECFE600043
:102CE40005F0EDFEDE0EEE6F000EEF6F2CEC10F033
:102CF400DE0EEC6F000EED6FB0EC0CF08AEC08F019
:102D0400900E1E01EC6F380EED6F000EEE6FC9ECE5
:102D14000CF0690E0001D36F000ED46FDE0E1E019D
:102D2400EC6F000EED6F60004DF3EEFE600051F3AA
:102D3400EFFE040EF06F000EF16F26EC0DF0010EA5
:102D44000001D325E96E000ED421EA6E6F00A7FFBF
:102D5400E9FF6F00ABFFEAFF6F00B9FFE0FE000E72
:102D64001E01E16F000EE16F670080FB01F0006A55
:102D7400600001F0E0FE600005F0E1FE60004FF34A
:102D8400D9FF600053F3DAFFDE500026000E012263
:102D9400600001F0E0FE600005F0E1FE600001F07B
:102DA400ECFE600005F0EDFEDE0EEE6F000EEF6F40
:102DB4002CEC10F0DE0EEC6F000EED6FB0EC0CF0AE
:102DC400D20E1E01EC6F390EED6F000EEE6FC9ECE2
:102DD4000CF0E60E1E01EC6F390EED6F000EEE6F77
:102DE400C9EC0CF0750E0001D36F000ED46F6000B7
:102DF4004FF3E9FF600053F3EAFF6F00B9FF1DFFD3
:102E040057EC01F0010E0001D325E96E000ED42128
:102E1400EA6E6F00A7FFE9FF6F00ABFFEAFF6F00E8
:102E2400B9FF1DFF57EC01F0020E0001D325E96E36
:102E3400000ED421EA6E6F00A7FFE9FF6F00ABFF1D
:102E4400EAFF6F00B9FF1DFF57EC01F0030E00010C
:102E5400D325E96E000ED421EA6E6F00A7FFE9FFC7
:102E64006F00ABFFEAFF6F00B9FF1DFF57EC01F0E5
:102E74008AEC08F060004DF3ECFE600051F3EDFEC7
:102E8400040E1E01EE6F000EEF6F85EC10F08AEC5D
:102E940008F0050E1E01EC6F390EED6F000EEE6F9B
:102EA400C9EC0CF0790E0001D36F000ED46FDE0E66
:102EB4001E01EC6F000EED6F60004DF3EEFE60003E
:102EC40051F3EFFE040EF06F000EF16F26EC0DF0DF
:102ED400010E0001D325E96E000ED421EA6E6F00C5
:102EE400A7FFE9FF6F00ABFFEAFF6F00B9FFE0FE49
:102EF400000E1E01E16F000EE16F670080FB01F020
:102F0400006A600001F0E0FE600005F0E1FE600090
:102F14004FF3D9FF600053F3DAFFDE500026000EB2
:102F24000122600001F0E0FE600005F0E1FE00C057
:102F340042F001C043F0600001F0ECFE600005F0D7
:102F4400EDFEDE0EEE6F000EEF6F2CEC10F0DE0ED9
:102F5400EC6F000EED6FB0EC0CF0910E1E01EC6FF7
:102F6400390EED6F000EEE6FC9EC0CF0060E026E1A
:102F7400670080FB00F0670084FB01F0025005E06D
:102F840001320032019EFF0FFAD700C04FF001C09A
:102F940050F02E0E1E01EC6F380EED6F000EEE6F2A
:102FA400C9EC0CF060003DF1ECFE600041F1EDFE77
:102FB400DE0E1E01EE6F000EEF6F2CEC10F0DE0E35
:102FC400EC6F000EED6FB0EC0CF08AEC08F0030E21
:102FD4001A6E000E1B6E496A4A6A0001D16BD26BED
:102FE4001E01E06BE16B1FD21E01BC8A7A0EEC6FEE
:102FF400370EED6F000EEE6FC9EC0CF0600009F1B6
:10300400ECFE60000DF1EDFEDE0E1E01EE6F000E13
:10301400EF6F2CEC10F0DE0EEC6F000EED6FB0ECE9
:103024000CF0AF0E1E01EC6F390EED6F000EEE6F5B
:10303400C9EC0CF08AEC08F0030E1A6E000E1B6E3D
:10304400010E0001D56F000ED66F790E1E01EC6FD4
:10305400380EED6F000EEE6FC9EC0CF07D0E000122
:10306400D36F000ED46F60004DF3ECFE600051F39B
:10307400EDFE140E1E01EE6F000EEF6F85EC10F0E6
:103084008AEC08F09A0E1E01EC6F360EED6F000EFE
:10309400EE6FC9EC0CF0000ECBB2010E1F011D6FD8
:1030A400300E1D2757EC01F08AEC08F08AEC08F08A
:1030B400400E496E000E4A6E0001D16BD26B520E67
:1030C4000B6E2B0E0C6E000E0D6E0D2EFED70C2EFD
:1030D400FCD70B2EFAD7000043504A5C02E1425061
:1030E400495CD8B097D000015050D65D02E14F50F2
:1030F400D55DD8B08FD0A3EC0DF0040E0B6EA80EE6
:103104000C6E0B0E0D6E0D2EFED70C2EFCD70B2E57
:10311400FAD700000000000E0001D81902E1010EE8
:10312400D71977E1010ED525006E000ED621016E68
:1031340000C0D5F001C0D6F0CBB24DD0710E1E0147
:10314400EC6F390EED6F000EEE6FC9EC0CF0600001
:1031540055F3ECFE600059F3EDFEDE0E1E01EE6F3A
:10316400000EEF6F2CEC10F0DE0EEC6F000EED6F26
:10317400B0EC0CF0870E1E01EC6F390EED6F000EF3
:10318400EE6FC9EC0CF0400E495C1E01EC6F000EB2
:103194004A58ED6FDE0EEE6F000EEF6F2CEC10F060
:1031A400DE0EEC6F000EED6FB0EC0CF08AEC08F064
:1031B400510E0001D36F000ED46F60004DF3ECFE8E
:1031C400600051F3EDFE400E1E01EE6F000EEF6F36
:1031D40085EC10F01ED0C10E1E01EC6F390EED6FA0
:1031E400000EEE6FC9EC0CF0600055F3ECFE6000CD
:1031F40059F3EDFEDE0E1E01EE6F000EEF6F2CECA8
:1032040010F0DE0EEC6F000EED6FB0EC0CF08AECFB
:1032140008F062D7BC8AD70E1E01EC6F370EED6F33
:10322400000EEE6FC9EC0CF0040E1A6E000E1B6E4D
:10323400A30E0B6E570E0C6E020E0D6E0D2EFED7E6
:103244000C2EFCD70B2EFAD70000EDD0BC8A5A0EF8
:103254001E01EC6F390EED6F000EEE6FC9EC0CF031
:10326400C50E1E01EC6F360EED6F000EEE6FC9EC4D
:103274000CF0800E01017E6F000E7F6F80EC10F069
:10328400BA866000F9F5ECFE6000FDF5EDFEE8ECB1
:1032940011F0BA86520E0B6E2B0E0C6E000E0D6ED4
:1032A4000D2EFED70C2EFCD70B2EFAD70000050EE0
:1032B4001A6E000E1B6E28EC10F0800E1E01EC6FCF
:1032C400000EED6FE8EC11F0300EAC12B50EAB6EE3
:1032D400D5EC0DF080EC10F0D00E0C6EC90E0D6E16
:1032E4000D2EFED70C2EFCD7000000004E0E1E0142
:1032F400EC6F390EED6F000EEE6FC9EC0CF0390E69
:103304001E01EC6F370EED6F000EEE6FC9EC0CF082
:10331400140E1E01EC6F370EED6F000EEE6FC9EC4C
:103324000CF0F50E1E01EC6F370EED6F000EEE6F14
:10333400C9EC0CF00001DB6BDC6B1D0EDC5D02E103
:103344004C0EDB5D25E2BA86820EDB25E96E010EAA
:10335400DC21EA6E6F00A7FFE9FF6F00ABFFEAFF15
:103364006F00B8FF00F0600001F0ECFE000E1E01DB
:10337400ED6FE8EC11F0020E0C6ED30E0D6E0D2EF7
:10338400FED70C2EFCD7BA960001DB4BDC2BD5D72D
:10339400800E1E01EC6F000EED6FE8EC11F028ECCE
:1033A40010F0020E0A6E450E0B6EAD0E0C6E050E7D
:1033B4000D6E0D2EFED70C2EFCD70B2EFAD70A2E2F
:1033C400F8D70000000077D72ED0000E1B1802E1BA
:1033D400000E1A18D8B458EF13F0000E1B1802E1AF
:1033E400010E1A18D8B40DEF14F0000E1B1802E1E8
:1033F400020E1A18D8B44CEF15F0000E1B1802E197
:10340400030E1A18D8B4F0D5000E1B1802E1040EEE
:103414001A18D8B41BD7000E1B1802E1050E1A188F
:0C342400D8B449D7D1D755EF13F0FFD72B
:1039EA0010EE1AF02E0E006E010E016E3F0EF66EEC
:0E39FA00360EF76E000EF86E85EC0DF0120022
:1034300020436F6E66696720626974203A205031BC
:10344000384632374B34325F466F73635F496E7470
:1034500065726E655F4C65676163795F696E7465FF
:103460007272757074735F313678345F504C4C5F94
:1034700036344D487A2E6366677363680D0A2046BA
:0F3480004F53433A36342E30204D487A0D0A0010
:10348F0020536F75726365203A2050494331384697
:10349F0032374B34325F4C6563745F5741565F620E
:1034AF00795F554152545F4354535F616E645F506F
:1034BF006C61795F62795F50574D5F5243325F3273
:0D34CF003032325F303930312E630D0A008B
:1034DC00204144435F496E69745F416476616E6359
:1034EC00656420283020E0202B56434320706F75F4
:1034FC0072203020E020343039352070747329204C
:10350C00204541313D5241313D706F746172200D47
:02351C000A00A3
:10351E002050726F746F636F6C65204861726477B0
:10352E006172652043545320737572206F757470E9
:10353E00757420524335202020626C6F63732064B3
:10354E006520646174613D36342062797465730D53
:02355E000A0061
:10356000204469726563746F7279203A433A5C5FF4
:103570004D696B726F435C5F4D657350726F6A6526
:1035800074735F4D696B726F435C5F3138463237DD
:0F3590004B34325F506C61795F5741560D0A0022
:10359F002050726F6A6574203A526561645F5741BB
:1035AF00565F616E645F506C61795F62795F5057EF
:1035BF004D5F31384632374B34325F323032325F03
:0B35CF0030392E6D637070690D0A002A
:1035DA002031384632374B3432205541525431204B
:1035EA003139323030206264732C20414443312017
:1035FA00313220626974732073757220454131201B
:03360A000D0A00A6
:10360D00204166666563746174696F6E2050494E22
:10361D002052433220E020536F7274696520505759
:10362D004D31207061722064656661757420210DC5
:02363D000A0081
:02363F00000089
:02364100000087
:02364300000085
:013645000084
:10364600603500D038009F35006D360030340048B4
:1036560038008F3400DA35001E3500B837005A3787
:013666000063
:02366700000061
:0236690000005F
:02366B0000005D
:10366D00204C65637475726520666963686965725F
:10367D0020574156202838626974732050434D29D4
:0D368D00207669612055415254310D0A002C
:10369A002041666669636861676520446174617385
:1036AA0020626C6F637320207369205242313D306F
:0B36BA00202D2D3E205242313D20000B
:1036C5002072652053746172742050574D31203833
:1036D50062697473206174203131303235206F6E28
:0836E50020524332200D0A00BF
:1036ED0020496E6974202050574D31202E2E537471
:1036FD006172742C202E2E2E73657420647574796E
:07370D003D3530250D0A00D7
:10371400202020204A6F7565206C652066696368E7
:103724006965722077617665203131303235204801
:053734007A200D0A00DF
:103739000D0A202D2D2D2D2D2D2D2D2D2D2D2D2D00
:103749002D2D2D2D2D2D2D2D2D2D2D2D2D2D0D0AE3
:01375900006F
:10375A002050574D312073757220736F72746965EA
:10376A0020524332203131303235487A200D0A0056
:10377A002045746170652033203B206C6563747545
:0F378A00726520646573206461746173203A0076
:103799000D0A4365206E2765737420706173207567
:0F37A9006E20574156202121212E2E2E0D0A0071
:1037B800204C4547414359206D6F646520666F7200
:0F37C80020496E7465727275707473200D0A005B
:1037D7000D0A2046696E206465206C6563747572F6
:0E37E70065206461746120776176650D0A00CB
:1037F5002D2D2D2D2D2D2D2D2D2D2D2D2D2D2D2DF4
:0E3805002D2D2D2D2D2D2D2D2D2D2D0D0A00AF
:1038130045746170652032202020466F726D61749B
:0B382300206368756E6B203A0D0A00F0
:10382E00204E6220646520626C6F637320363420F4
:0A383E00627974657320203D2000BC
:1038480020456570726F6D3A206E6F7420757365D0
:0938580064202E2E2E2E0D0A0014
:10386100204669636869657220574156666D742008
:08387100202E2E4F4B0D0A0022
:103879000D0A20726573746520647520426C6F634C
:07388900202331200D0A008D
:103890004672657120456368616E74696F6E6E6112
:0638A0006765203D2000D9
:1038A6000D0A2050726573656E746174696F6E20BF
:0538B6003A200D0A009C
:1038BB0020476C6F62616C2046696C652073697A76
:0538CB0065203D200016
:1038D000204D696B726F432070726F20372E363027
:0338E0000D0A00CE
:1038E3002046696368696572205249464620210D66
:0238F3000A00C9
:1038F500204E622064652063616E617578203D000D
:10390500205461696C6C652044617461203D200020
:103915003031323334353637383941424344454600
:0F392500205461696C6C6520426C6F63203D001B
:0E39340020466F726D61742050434D203D009F
:0C3942000D0A205265E775203A0D0A00BE
:0C394E002045746170652035200D0A00D2
:0C395A002045746170652034200D0A00C7
:0B39660020454131206D6F79203D00AD
:0B3971000D0A20426C6F632023200031
:0B397C0020496E64657831203D20007A
:0A398700204F66667365743D200052
:0A399100206279746573200D0A00AE
:0A399B00206279746573200D0A00A4
:0A39A500457461706520310D0A00C1
:0939AF002042797465730D0A00D1
:0939B80057415645666D7420006C
:0939C10020426C6F6320232000FA
:0839CA00203B54656D703D00C7
:0639D20020487A0D0A00F6
:0539D8005249464600C3
:0539DD0020B0432000B2
:0439E200206A3D001A
:0339E600203E0080
:020000040030CA
:0A000000772BF7BF0B3F9F2F010085
:00000001FF
